:020000040202F6
:10A0000000FC02029DA6020205A3020205A30202B1
:10A010000000000000000000000000000000000040
:10A0200000000000A0CF0202E8CF020205A3020256
:10A03000000000000000000005A30202B5A8020213
:10A04000A7A1020205A3020205A30202BDA6020205
:10A0500005A3020205A302029DA2020235A3020289
:10A0600005A3020205A3020205A3020209A302023C
:10A0700005A3020259A9020205A3020205A30202D6
:10A0800005A3020205A3020205A30202DDA8020243
:10A09000F9A8020205A3020205A3020205A3020217
:10A0A00019A9020223A90202A9A1020205A3020220
:10A0B00005A3020205A30202000000000000000048
:10A0C0000348854600F040F8004800470DC20202F0
:10A0D00000FC020230B50B4601460020202201247C
:10A0E00009E00D46D5409D4205D31D469540491BCC
:10A0F0002546954040191546521E002DF1DC30BD15
:10A1000003460B439B0703D009E008C9121F08C090
:10A11000042AFAD203E00B780370401C491C521E3B
:10A12000F9D27047D2B201E00270401C491EFBD246
:10A1300070470022F6E710B513460A460446194652
:10A14000FFF7F0FF204610BD064C0125064E05E046
:10A15000E36807CC2B430C3C98471034B442F7D348
:10A16000FFF7B2FF88CD0202A8CD020230B58C18ED
:10A170000278401C13071B0F01D10378401C120901
:10A1800006D10278401C03E005780D70401C491C84
:10A190005B1EF9D101E00B70491C521EFBD1A1429C
:10A1A000E6D3002030BD70477047B0B5044645186F
:10A1B0000020AC4205D2217880B200F0B7FB641CCD
:10A1C000F7E780B20024214600F0B0FB214600F002
:10A1D000ADFBB0BD10B504210A060AD0027852B218
:10A1E000D3091B241C40520062400270491E401CCF
:10A1F000F2E710BDB0B501230022D4B20355DCB2A2
:10A200000A555C005C401B06DD171B232B40634096
:10A21000DCB2521C012CF0D10178FF228154B0BD78
:10A22000F0B500210E4A0B46002B0C4605D030CA73
:10A23000ED5CFF266E40A45D083A63256540042668
:10A24000370606D06700E4B2E4093C196540761E83
:10A25000F6E7C5545B1C01242402A342E4D1F0BDFF
:10A26000F4E9020270B5002213461446E5B2465DD9
:10A27000B34204D06C1CE5B2A542F7D000E0CC5448
:10A280005B1C01242402A342EFD170BD0B78037044
:10A29000491C401C521E1306F8D17047BCB5184C1F
:10A2A00020680568002001A90870C0B2082825D2DE
:10A2B000012211048140294209D0226851608000A6
:10A2C0002018826A002A16D001A8012112E0130288
:10A2D00083402B4201D0022104E082402A420AD06E
:10A2E0000321134622685360800020188268002AE8
:10A2F00001D001A890470198401CD4E7BCBDC046DE
:10A300001CE80202FEE7000010B509480168CA69AE
:10A3100020231343CB610269032A08D1012293054C
:10A320000C689C430C605102C26E0A43C26610BDA9
:10A3300084E80202F8B50C4806460C360068876BC4
:10A340000024122C0ED00125A5403D4207D03168D3
:10A35000002904D020468847034800688563361DDD
:10A36000641CEEE7F8BDC04600E9020210B501200A
:10A37000440619200203C0492046FFF7C1FE2068A9
:10A3800080F30888606800198047002010BDC0462F
:10A39000F0B585B000900025144E0A202C46002808
:10A3A00021D00290039108463146FFF793FE0746FD
:10A3B0003030009948550195FDB204942543681E3C
:10A3C0002C46844177430A213046FFF783FE064638
:10A3D000002D01D0019D6D1C02AB0BCB1B191C463F
:10A3E000C91B401EDBE705B0F0BDC04600CA9A3B62
:10A3F000FEB50C460546E031102200F0BBFA019490
:10A40000D0340D27284600F077F810222846029411
:10A41000214600F08BF800200424210606D0C6B2A5
:10A42000A81900F011F8641E301DF6E7029C103CDC
:10A430007F1E3806E6D1284600F05EF81022284636
:10A44000019900F073F8FEBDF0B58BB00446C078FA
:10A450000890A07802902778049765780795254E94
:10A460002046B04760780990A0780690E078019087
:10A4700020780A902046B0473146A0780590207891
:10A480000390E07800906678204688473946694016
:10A490006078A2784240E3785340207858400246E2
:10A4A000029B5A404A400A9D6A40019F7A40009DA3
:10A4B0006E407240E270089A50404140069D6940EB
:10A4C0007940039F059A57407940A1700146594051
:10A4D000049A5140099A514069407140617007994E
:10A4E000484058400A9948405040784020700BB08E
:10A4F000F0BDC046D5A10202417B427A4273427947
:10A5000043784371427241708178827A827081729D
:10A510008179827B82718173C178C279C270C27A7B
:10A52000C271C27BC173C27270470000B0B5064BE6
:10A5300004781C5D0D7865400570491C401C521E56
:10A540001406F5D1B0BDC046E2EC0202F0B587B00A
:10A5500004460120019005902F48202221460378CF
:10A560002370401C641C521E1306F7D140393D3144
:10A5700006A80422FFF78AFE3F20C0430490202152
:10A580000294EF2945D86518049C20341C2008400B
:10A590001028039121D0002823D1009506AD6878BA
:10A5A00006992870A878EA78AA706870E97004267D
:10A5B0002846314600F070F905AF2846009D39461F
:10A5C000324600F0D7F9019A50B2C0091B21014070
:10A5D00052004A4001923A7003E006A8042100F0BC
:10A5E0005BF904982F462D1806AE04223046294602
:10A5F00000F0C0F906983855707821216854B07879
:10A6000022216854F078232168540399091D029C83
:10A61000B7E707B0F0BDC04614CD0202F8B500F0B0
:10A6200071F800281FD16C461148208001273A0399
:10A630000025104E2846314600F0F2FF1036022366
:10A6400028463146224601F02FFC7C0619200203E1
:10A6500009492046FFF754FD206880F308886068A8
:10A6600000198047F8BD0A2000F066FD00F004FBE9
:10A67000FFFF000000D0020400A0000470B50546F2
:10A680004E1C0024761E05D0284600F087F80128CD
:10A69000F7D100E0E443204670BD000006480168A1
:10A6A000032291430160016801220A43026000F025
:10A6B0000DF901F0A7FEC0462800004080B50B4907
:10A6C0000868002800D480BD094802680423032AD2
:10A6D00001D01A4300E01A460A6006490A68002AB7
:10A6E000F1D041680020904780BDC0462C10014049
:10A6F00000E802024CF2020280B500F05BF8002094
:10A7000080BD0000FEB568460026068101960096D1
:10A710003320FFF7F1FF114800F038F90446012813
:10A7200012DB0F480F4FB8470F48B8476D46284611
:10A730002146FFF72DFE0DA0B8472846B8470EA0CA
:10A74000B84710A0B84706E00220C043844201D3B6
:10A75000664200E00426F0B2FEBDC04668F2020286
:10A7600034CD0202D9A70202E2EA02020A0D205306
:10A77000697A653A200000002042797465730D0AF9
:10A78000000000002D2D2D2D2D2D2D2D2D2D2D2DAD
:10A790002D2D2D2D2D2D2D0A000000000D49896C29
:10A7A0004A69D20501D40020704749680170012030
:10A7B0007047C046E0B501A908700648806C416A40
:10A7C0000029FCD101A901200023024602F048F82B
:10A7D0008CBDC04654E9020210B50446207800281A
:10A7E00003D0FFF7E7FF641CF8E710BD70B50278EF
:10A7F000302A27D1427820231343782B22D1827824
:10A80000002A47D05622D343002402220B2A41D0EB
:10A81000855C002D31D02E46413E062E02D21E46CA
:10A8200020360AE02E46613E062E1E4605D32E46F1
:10A83000303E092E1FD81E462736751924012C19C3
:10A84000521CE3E7002213460B2A23D0845C002C21
:10A850001CD04B2C17D04D2C11D06D2C0FD06B2C45
:10A8600011D02546303D092D05D80A255D432B1909
:10A87000303B521CE8E700200AE00C6007E0002AA9
:10A8800008D01B0502E0002A04D09B020B600120C7
:10A890000B2A00D3002070BD10B5054A03789468D8
:10A8A000E35C0370401C491E0B06F7D110BDC04687
:10A8B000F4E9020280B504480168491C016000699E
:10A8C000002800D0804780BD50F2020201480249B2
:10A8D000016070470CE802020026B803E0B50D499C
:10A8E00008680022C2600192CA68002A02D001688A
:10A8F00001A890478CBDC046E0B506490869002212
:10A90000C26001220192CA69002A02D0016801A82E
:10A9100090478CBD64E8020280B5002001F040FE43
:10A9200080BD80B5012001F03BFE80BDB0B50123A4
:10A930001A028A18D903074B44001506ED0F2C198B
:10A94000084200D05C40204654000A422246F3D020
:10A9500080B2B0BD21100000E0B500200190044895
:10A96000C268002A02D001A8002190478CBDC046D1
:10A97000E4E9020210B50B7804785C400470491CCD
:10A98000401C521E1306F6D110BD0000F0B585B074
:10A99000044600F089F9B24D002702200090A880FB
:10A9A0006F80B048E8602F616F61AF610120019056
:10A9B000000504900394EF612F626C62384602F048
:10A9C000B3F8AF6228460499FFF758FE002810D06C
:10A9D0006869A969012901DB401C6861062800DB60
:10A9E00004E14320FFF7E6FE039C286A0028E5D037
:10A9F000F8E0287801280CD002289B4A0CD00428C3
:10AA000040D0182865D0412800D1F7E06128DFD177
:10AA1000F4E08026944A01E001998E02107005242A
:10AA200034430120E88080B28F49844208D9081855
:10AA30000499FFF723FE0028CAD1E888401CF1E7FB
:10AA40008878FF2242404978914200D0D6E0688859
:10AA5000884203D02978012900D0CFE0401C6880CB
:10AA6000814CE01C3146FFF7A0FB04213143615CBF
:10AA700003223243A25C12025118814200D0BDE091
:10AA8000AE6200E0AE6A00246C61002E00D1A3E04B
:10AA9000701C00D1CFE074484178E869C2B291429D
:10AAA00023D1002845D0686A6F49C91C3246FFF798
:10AAB00027FB03986863AC63AB6A9C4217DA2946AC
:10AAC000443100F00DF9686B10306863AC6B1034E2
:10AAD000F1E728460499FFF7D1FD002800D077E779
:10AAE0002878182800D073E79FE015207AE7688857
:10AAF00080025E494018039AEA632864E9680026E8
:10AB0000304601F0D1F9002800D083E0296CE868D4
:10AB1000884202D0AA6891427CD9A96A0818E860E4
:10AB20000620FFF747FE52480660A888401CA88010
:10AB30004CE04D4BD87800287FD00020D91CE8622B
:10AB4000296301991A1800290AD0FF2808D8D1785A
:10AB5000484C2154401C111DE86229631179F1E72A
:10AB60000021444B1954101DE9622863009AD24316
:10AB70000292425C202A0FD00E290DD842186B1881
:10AB8000521C029CA418A4783E465427DC55374634
:10AB9000491CE9622A63ECE72846543000224254FB
:10ABA000491CE96229460831FFF720FE19200203FB
:10ABB000501CA968814248DC00202A4900F030FD81
:10ABC0000620FFF7F7FD4320FFF7F4FD0198A86189
:10ABD000E869401CE86107E70620FFF7EBFD01206C
:10ABE0002862039C286900282DD1E4E61825284610
:10ABF000FFF7E0FD2846FFF7DDFD08E018242046BA
:10AC0000FFF7D8FD2046FFF7D5FD0098C74338462B
:10AC100005B0F0BD18242046FFF7CCFD2046FFF715
:10AC2000C9FD0098C043471CF1E700206861009807
:10AC3000C043801CA8620620DDE70620FFF7BAFDAE
:10AC4000012028612862AF68E1E718242046FFF759
:10AC5000B1FD2046FFF7AEFD0298871CD7E7C0463E
:10AC600008EA020200A0000444EE0202009C000474
:10AC700068F70202E2EA0202BFF34F8F084809496F
:10AC80000160BFF34F8F00BFFDE7C046BFF34F8F9A
:10AC9000034804490160BFF34F8F00BFFDE7C04682
:10ACA0000CED00E00400FA0570B51C4E0A4C0B4D8B
:10ACB0003560746028462146FFF79CFA1648B0605C
:10ACC000FFF7AEFAF5602846FFF740FC3461B06844
:10ACD0002146FFF7C7FA70BDE2EC0202E2EB020286
:10ACE000F8B50C460746FFF7DFFF0B4D1026284648
:10ACF00039463246FFF7CAFA0848C1683846FFF7B6
:10AD000077FB384621463246FFF734FE2046294677
:10AD10003246FFF7BBFAF8BD68F60202F4E9020218
:10AD200070470000F8B516484C210160FF2402343A
:10AD3000144F2046B847322000F005FA00F0DCF846
:10AD40000125284600F0E2F8284600F033F800F02C
:10AD5000CDF80D48B84700263046314600F09EF940
:10AD60002846314600F09AF93046B8470220B847E5
:10AD70004734204601F04AFB01F064FBF8BDC046B1
:10AD8000480000401DAF02020102000070470000B1
:10AD9000B0B505200424064D2146A84706202146CB
:10ADA000A84701202146A8470E202146A847B0BD4C
:10ADB000BDC1020202490A6802408242FBD17047CB
:10ADC00004600040B0B53C4801688A073B4C07D599
:10ADD00001797F221140E36993435918E1610168C9
:10ADE000890407D55E21405C7F210840226A8A439E
:10ADF00010182062172000F0F7F83148016802228D
:10AE00000A4301218A4302602E482F4901602F48DE
:10AE10000021C17181791F2529408171817A427C8D
:10AE2000837C1B029A18C37C1B04D218037D1B066B
:10AE3000D218274B9A4218D1427B837B1B029A1867
:10AE4000C37B1B04D218037C1B06D218214B9A42E9
:10AE50000BD1C27A037B491E122906D81902891820
:10AE60001D4A914201D1202101720178CA0602D106
:10AE70001022114301702068202188432060264859
:10AE80001649016041680029FCD501F0A7FA0A21A2
:10AE9000C841032800D8FEE71148C1680F2291433A
:10AEA000C16001680F4A0A400260192000010E4982
:10AEB00048600D60B0BDC046E4ED02022C000040C9
:10AEC000040200400C060040AF6B100A6B0001400A
:10AED0004D383650312E323607340000FE1C0080CB
:10AEE000C8600040FEFFC3FF0C04004080B517207F
:10AEF00000F072F8002080BD10B51724204600F045
:10AF000073F8204601F070FA002010BD0121C90736
:10AF1000014301480160704700600040B0B5C2B213
:10AF2000000AC1B2022A0CD0012A12D0002A2CD168
:10AF30008A1E3148022A19D20122032926D051043F
:10AF400025E02D48426800291BD0014620390A43DC
:10AF50001AE0294C2568C81E02280ED3012926D0E4
:10AF600000292DD101208007854330E0002914D12C
:10AF70000121490702688A4317E004291DD00220F5
:10AF80001CE0012189078A434260B0BD11040322FD
:10AF90001204C36A93435918C1620E490A689207A2
:10AFA000FCD50121490702680A430260B0BD0520B3
:10AFB000000785432046203808E0012000F09EF875
:10AFC000044801684906FCD50520000705432560B3
:10AFD000B0BDC0462C0200400121814006480268F5
:10AFE0008A4302607047C0460121814002480268DE
:10AFF0000A4302607047C0462000004080B500F060
:10B000003BF83D4909688900890FC84080BDC046AA
:10B0100080B5FFF7F3FF384909680901890FC84077
:10B0200080BDC04610B505280AD8C04678440079CE
:10B030004000874402070F0A121700F01DF810BDE8
:10B04000002010BDFFF7DAFF10BD012081074A6A1A
:10B05000520004D5FFF7DCFF10BD01208107096A0B
:10B06000C00310BD0120840700F006F8616A0903DF
:10B07000890FC84010BD000001218807026A006ADC
:10B08000C00001D5044800E00248520000D4C803C3
:10B090007047C046006CDC020026B803042829D89B
:10B0A000154AC046784400794000874402091017C9
:10B0B0001E0003200007136883438807800812E0FE
:10B0C0000320800613688343880700090BE00320F0
:10B0D0008004136883438807000B04E0FF2000020C
:10B0E000136883430802181803E01068FF2398438D
:10B0F000401810607047C0462400004009490A68A3
:10B10000094B1340000418430860084800210160FF
:10B110000749084A0A600D21490242680A43426011
:10B120007047C0464800004080FFFCFF100200400E
:10B1300004010040FF0F000080B57D21C900484395
:10B1400000F001F880BD00280AD030B407252C0299
:10B15000CD256419604340091238001FFDD830BC6A
:10B1600070470000F8B505460120072D66D80C464B
:10B17000002963D0444F38680169C90736D10526D4
:10B180003046FFF731FF304601F02EF903CF036957
:10B19000012213430361002918D403200B46834383
:10B1A0006D481E588807C00EFF278740BE434027C2
:10B1B0008740374368481F501F2008408240674837
:10B1C000026067480260304800680FE08A07D20ECC
:10B1D000FF2696400F230B40083B03218B435D491C
:10B1E0005F58B743402696403E435E506901401881
:10B1F000012109024218E369DB069B0CA569ED00F9
:10B20000EDB2EB18536062685207520B23685B077C
:10B210005B099A18A3685B079B0CD218E3685B076D
:10B220005B0DD21823695B01DBB2D21863699B07FF
:10B23000DB0ED2188023134343500020F8BDC046D4
:10B24000F8B505460835104C2668F668EE40F50757
:10B2500001D00220F8BD069D8600A619B560400108
:10B2600024682018009301231D02461977680724DB
:10B27000A7437760F16032610099B1604159194389
:10B2800041510020F8BDC0461CE8020200013A49C5
:10B29000085840687047C046F8B505460120012DA2
:10B2A00045D80C46002942D0002D03D0012D04D1F1
:10B2B0000F2000E00E20FFF797FE29012E4843588B
:10B2C0000020D86027686568A668F607B60FAD0746
:10B2D0002D0FAE192569EA07920EB618022F04D079
:10B2E000012F03D10122164300E040369E60E26840
:10B2F0001A60214A51188D606269CA604968002944
:10B3000016D403220B469343134A9C588D07ED0E27
:10B31000FF26AE40B4438026AE4026439E501F22F7
:10B320000A40012191400D4A11600D4A1160F8BD9B
:10B330008A07D20EFF2494400F230B40083B0321C1
:10B340008B4304495D58A543802494402C435C50B2
:10B35000F8BDC0461CED00E000E400E080E200E043
:10B3600000E100E00001044A105801608168802279
:10B370000A4382607047C04664E80202F8B50E4690
:10B380000446032100F0F8FB0546002838D120468A
:10B3900000F09CFB0621204600F00AFD7C20604363
:10B3A000EC490F183A6A5643BA69B21808588260D5
:10B3B000172179563E461736002909D5C169202242
:10B3C0000A43C2610121F966890502680A430260E5
:10B3D0000521204600F0ECFC307840B200280FD464
:10B3E000084800687D26F100FEF774FE71014143B4
:10B3F000204600F0E5FB204600F040FD01203861CA
:10B400002846F8BD64F20202FEB5064602907C2092
:10B410007043D0490F18FD6EECB2601E02280BD2AB
:10B4200028040121000E28D03046019100F03EFB97
:10B430000199C00705D020E0032C1BD12804000E81
:10B440001AD038466C302D0C002101910160304635
:10B4500000F014FDE9B20120002902D0032900D038
:10B46000062038613A6F002A02D002A82146904790
:10B47000019902E0002100E001210846FEBDC0461E
:10B48000F8B50C460078B34DE96881422BD1032C06
:10B4900052D1686EA96E88424ED9002406212046FA
:10B4A00000F086FC2868E96D81602046214600F0A6
:10B4B0007FFC2E4660364CCEE8682968AC8C264F5F
:10B4C00000979B1BA34200D81C46A3081431FFF72A
:10B4D000B7FEA86E0019A866286E00192866E86DE8
:10B4E0000019E865F8BDA968814224D1032C26D152
:10B4F000E88CE96D0918E965296E09182966A96EB5
:10B500000818A866696E814219D9002406212046D0
:10B5100000F04EFC2868E96D81600121204600F0B2
:10B5200047FC296EA868EB8C2A680B4C00941432F7
:10B530009B08FFF785FEF8BD002000F0C7FA012048
:10B54000C1072A6813688B431360E96E22040A431B
:10B5500000021043E866F8BD81B40202BCB5007871
:10B56000F24DAA68824237D1032929D1686DA866B5
:10B57000AA6DAB6A1B18EA652B66AA6C521CAA64FA
:10B580006A6E82421CD9012000025E30FFF7DBFDAB
:10B59000686CA96C022920D381421ED1E88C696DA8
:10B5A0000818686500240621204600F001FC286880
:10B5B000E96D8160296D204600F0C0FD2B6D24E00F
:10B5C0000120C2072B681C6894431C60EA6E0904C2
:10B5D000114300020843E866BCBD0229FCD3814246
:10B5E000FAD2E88C696D09186965A96D0818A86513
:10B5F00000240621204600F0DBFB2868E96D81600D
:10B60000E98C204600F09AFDEB8C296EA8682A6828
:10B61000024C00941432FFF713FEBCBD5DB502026C
:10B62000F0B587B004460127880E6AD01546002A77
:10B6300067D00E468120C004401B884261D37C2025
:10B640006043BA4908180590818C30460691FEF790
:10B6500041FD002955D128460699FEF73BFD0029FA
:10B660004FD105988069361A30460699FEF732FDAB
:10B670000746039670190190069E3146FEF72AFD93
:10B680000546C01B04900598006A02903146FEF7FB
:10B6900021FD049981420CD2AF4231D22046394675
:10B6A00000F022FA2046FFF7AFFE0028FAD17F1CF7
:10B6B000F2E705900398029E3146FEF70BFD054622
:10B6C000304668430399081A0198314600D06D1C32
:10B6D000059E6E43FEF7FEFC0490029941430198DB
:10B6E000401A03900699B7420ED22046394600F020
:10B6F000FBF92046FFF788FE0028FAD17F1CF1E70E
:10B700000027384607B0F0BD0398FEF7E3FC064675
:10B71000049FBD420AD220462946FFF72FFE20464D
:10B72000FFF772FE0028FAD16D1CF2E70598784306
:10B73000059000273D46B542E3D2059829182046DA
:10B7400000F0D2F92046FFF75FFE0028FAD16D1C09
:10B75000F1E7C04684E80202F8B5002801D00124D0
:10B76000B0E07826DF4FB85D002801D00024A9E0C2
:10B77000002904D0384614301422FEF7C1FC0024FE
:10B78000FC6615252846FFF72FFC284600F02CFE06
:10B79000204600F09BF9B88AB97D0907090B091802
:10B7A000F87DC207D20889188207D20F520589187E
:10B7B000C206D20FD20589184207D20FD2068918C5
:10B7C0008206D20F520789180007C00F800708436E
:10B7D000396808600A21204600F0EAFA3220FFF7B3
:10B7E000B2FC0821204600F0E3FA20212046224640
:10B7F00000F0FAF93868017D0A46C23A53425341D3
:10B800007422BB54027D007DC22903D1F97D012041
:10B81000084014E000240321204600F0C9FA20214A
:10B820002046224600F0E0F93868007D42080120F9
:10B830001040F97D0A43D20701D0014004D0012114
:10B840004140002000F042FC7720385C012803D101
:10B8500002200021FFF722FC0024204600F00EFB0E
:10B860001720385600282AD57868002817D40321D5
:10B8700002468A43154953588507ED0EFF21A9401A
:10B880008B438021A9401943104BD1501F21014007
:10B89000012088400E4908600E4908600FE08107CA
:10B8A000C90EFF238B400F220240083A0320824337
:10B8B000054815589D4380238B402B43135001208E
:10B8C000B85538612046F8BD1CED00E000E400E00A
:10B8D00080E200E000E100E0FEB51E46174602915E
:10B8E00005460621019100F063FA7C246C43CB48A5
:10B8F00000590299816002952846314600F01EFCED
:10B90000C6480019002E05D03978026811757F1CD1
:10B91000761EF7E7974800687D21C900FEF7DAFB3D
:10B9200001994143029800F04BF9FEBD84E8020200
:10B93000F0B58FB004460126880E00D1B0E01D4658
:10B94000002B00D1ACE00F4604928120C004401BC4
:10B95000884200D2A4E00221204600F00DF90646FC
:10B96000002800D09CE00397204600F0AFF87C2030
:10B970006043AA490F18F87D4006029528D4069422
:10B9800028463D462435B98C0191FEF7A3FB05906E
:10B9900000240598844257D20621069800F008FA40
:10B9A0002888604303994018396888600026069803
:10B9B000314600F0FDF9049A2888864206D2604399
:10B9C00010183968097D8155761CF5E7641CE0E79D
:10B9D000032000260399F96504993A46603262C251
:10B9E000F8660120C00739680A6802430A60062128
:10B9F000204600F0DDF93868039981602046314621
:10BA000000F0D6F907AD284920222846FEF778FB3A
:10BA1000BC8CF8682946029DFFF7A4FBF8683968DA
:10BA2000E14A0092AC4200D32C46A3081431049A98
:10BA3000FFF706FCB86E0019B866386E0019386654
:10BA4000F86D0019F8652BE00598019941430298BB
:10BA5000441A1BD00621069800F0AAF928880599F7
:10BA60004843039940183968886000260698314693
:10BA700000F09EF9049AA64208D228880599484306
:10BA800080193968097D1154761CF4E7069C20461C
:10BA900000F01CF8204600F0F1F901203861002682
:10BAA00030460FB0F0BDC046F8CB020210B50446D8
:10BAB000022100F07DF920210022204600F094F8B8
:10BAC0007C206043F6490858007D10BD80B57C217C
:10BAD0004143F34A52581021D1610A4600F084F8DC
:10BAE00080BDC04684E80202F8B50E460446032134
:10BAF00000F042F80546002839D12046FFF7E6FF5E
:10BB00000621204600F054F97C206043E4490F18D8
:10BB1000BA8C5643BA69B218085882601721795610
:10BB20003E461736002909D5C16920220A43C26161
:10BB30000121F966890502680A4302600421204652
:10BB400000F036F9307840B2002810D497480068E9
:10BB50007D21C900FEF7BEFA4B21C90041432046B2
:10BB600000F02EF8204600F089F9012038612846BF
:10BB7000F8BDC04664F2020270B50123EFF31082F3
:10BB80001A4002D1EFF3108472B67C244443C448B7
:10BB9000041926690020062E0DD81D46B540EE0674
:10BBA000760F04D16126354203D0184603E0022007
:10BBB00001E010342160002A00D162B670BDC04699
:10BBC00070B50C46054600F037FC06462846FFF7E0
:10BBD0006DFFC00707D06420FFF7B5FA00F02CFC1A
:10BBE000801BA042F2D970BDF8B500920D467C21B1
:10BBF0004143AB4844182746143700F01DFC064665
:10BC00002068C06928400099884205D100F014FCE2
:10BC1000801B39888842F3D9F8BDC04684E8020207
:10BC2000F0B591B01F460D460123890E00D1B5E055
:10BC3000002F00D1B2E08121C904C91BA94200D262
:10BC4000ACE0079306927C22424395498E180890F7
:10BC5000F48C28462146FEF73DFA002901D0079BC7
:10BC60009CE038462146FEF735FA0029079B00D0B4
:10BC700094E004210898FFF77FFF0346002800D0D6
:10BC80008CE030462630B169059107900488089809
:10BC9000FFF71CFF0598281A04902146FEF71AFAB0
:10BCA00005900498C0192146FEF714FA0290F07D21
:10BCB00040063BD43046183001900025079C05987B
:10BCC0000299884264D227880621089C049505467B
:10BCD0002046039100F06CF80798008805956843AA
:10BCE000049D019909684018316888600121204647
:10BCF000079C00F05DF86F430698C0192188002961
:10BD000005D0027833681A75491E401CF7E72748AA
:10BD100000687D21C900FEF7DDF9039941430898C9
:10BD2000FFF74EFF6D1C0598401CC9E7022000225A
:10BD3000F565069931667766B2661746F0660125A5
:10BD4000E80731680A6802430A600621089C204619
:10BD500000F02EF8F06D316888602046294600F02A
:10BD600027F809AC0F4920222046FEF7C9F9B06830
:10BD70002146FFF7F7F9B068316E079A13883268E9
:10BD8000094C009414329B08FFF75AFA3B4605E031
:10BD9000089800F073F8012030610023184611B0B4
:10BDA000F0BDC046D8CB020281B4020264F20202A6
:10BDB000F0B587B00D46044601210A46FFF714FF8F
:10BDC0000227204639463A46FFF70EFF1423039513
:10BDD0006B43DC206043284908180590C018068A88
:10BDE0008568C17C06917C2104946143EB4A52181A
:10BDF0007424145D012C12D102970196039E012E2A
:10BE000000D00295012EE54F01D138240694752407
:10BE1000125D012A019C029D04D0224603E03246B5
:10BE2000DE4F03E00322072E00D02246069EDC4CA4
:10BE300014403606AD07ED0AAD192C19059DEB58D7
:10BE4000DB075B0CE4184368DD072D0C6419857C67
:10BE50006D076D0B6419C0684007000A20187958F7
:10BE60004860002A06D0012B04D102210022049848
:10BE7000FFF7BAFE07B0F0BD38CC020210B5044699
:10BE800001210A46FFF7B0FE022120460A46FFF7CD
:10BE9000ABFE7C206043C14908580249816110BD56
:10BEA00084E80202000093EBF0B593B00546012749
:10BEB000880E00D102E11E46002B00D1FEE00C46A8
:10BEC0000A928120C004801B884200D2F6E004213F
:10BED0002846FFF751FE0746002800D0EEE07C2000
:10BEE00009956843AD4902900F18BC650021079180
:10BEF0007965701E06900019B964B9690391621AD8
:10BF00000A99B962FC623863104605927A63F98C2B
:10BF10000891FEF7DFF80546B863069805990818FA
:10BF20000899FEF7D7F80695411B4A1C3B463C335F
:10BF300007C3079A002931460AD0089D6843311982
:10BF4000039BC91A0A1A06996943181B401941181C
:10BF50003D4648353846583006903C465434F964DE
:10BF60003A650998FFF7B2FD39464C31F87D400635
:10BF70000497079150D43E464436394640310891E3
:10BF8000394626310391503705970120069F0296C6
:10BF900028603368984200D989E008990968012926
:10BFA00007D000290ED120680A990A183968079825
:10BFB00023E0012808D0984223D120680A990A1862
:10BFC000396819E0012811D120680A990A183968DE
:10BFD000079F3B680998FFF77FFC3868069F396820
:10BFE000091839602168081820600AE021680A9A57
:10BFF00052183968984207D1059803680998FFF7E5
:10C000006BFC2868401CC3E7039E33880998FFF740
:10C0100063FC3088029EE2E70BA80A90294920229F
:10C02000FEF76EF802985D49085801680122D207B0
:10C030000A430260B8680A99FFF794F802200A9050
:10C040000027069B19680498826AC16502664666E5
:10C0500087660A99C166079E3068216809182160C1
:10C0600029684A1C2A601A6810181860002925D10E
:10C07000049D294660310A912E465C362C460834D0
:10C0800006210998FFF794FE286831688160079EB1
:10C090003168099800F052F833680A9801682068FE
:10C0A0002A68094C00941432FFF7CAF806E0099890
:10C0B000FFF7E4FE0120049908610027384613B019
:10C0C000F0BDC046B8CB02025DB50202B0B50D4668
:10C0D00004460621FFF76CFE07212046FFF768FEA5
:10C0E0007C2060432D4909187420085C012811D177
:10C0F000681E8541AA010868027500220275752232
:10C100008A5C012A0ED114307622895C4A424A4167
:10C11000510006E0086800210175691E8D41690023
:10C1200014300170D94800687D21C900FDF7D2FFA5
:10C13000282141432046FFF743FDB0BD70B50D46B1
:10C140000446012631463246FFF74EFD02212046C5
:10C150000A46FFF749FD7C20604310490A18742302
:10C16000D25C012A01D0F30400E033050C4E2E40CE
:10C17000F318012A02D01922520601E00722D20642
:10C180009A18084BD21808584260002D04D002219A
:10C1900000222046FFF728FD70BDC04684E8020259
:10C1A000FF3F00000080800010B501242046FEF70C
:10C1B0001BFF204600F018F9002010BD124A072886
:10C1C00009D880000F2383408140194010689843AC
:10C1D0000843106070470F280AD8800020380F23CA
:10C1E000834081401940506898430843506070472D
:10C1F000800040380F238340814019409068984365
:10C20000084390607047C046340000408AB0FEF793
:10C2100089FDFEF7BDFDFEF7D5FD0024204600F0A8
:10C2200013FC5049204600F031FCFFF7BDFFFEF73C
:10C23000ADFD02AD4C4920222846FDF761FF2046A6
:10C240002146FFF789FA01242046294600F062FAC8
:10C2500046A0FEF7C1FA009467064D4E594D0024E2
:10C26000204600F061FC01AA1680022320464749BF
:10C27000FFF75EFB0020FFF7C7F80028FAD101A8FE
:10C28000008844490880444988420AD0434988428A
:10C290001BD0B0420CD14DA0FEF79EFAFEF7BEF9BE
:10C2A000DDE73FA0FEF798FA3846FEF75FF8D6E7DD
:10C2B0001920020338462946FDF722FF386880F32B
:10C2C00008887868C0198047C9E739A0FEF784FA62
:10C2D0001920020300202946FFF7A2F9FEF7E4FC2B
:10C2E0000098C6042B4F1237700C042823D8002066
:10C2F000642331463A46FFF71BFB00242046FFF734
:10C3000083F80028F9D1632C07D822490819123084
:10C31000891CFEF7E5FC1034F5E70020642329466C
:10C320003A46FFF77DFC0020FFF76EF80028FAD1AF
:10C3300064356436D8E701AC234820800025022606
:10C340002846124F39463246FFF76AF928463946E1
:10C3500022463346FFF764FC7D208000FEF7ECFEAA
:10C36000FEF794FC10E8020218CC02024D4B383064
:10C3700030302D426F6F744C6F616465722D563191
:10C380002E31C6F4B6AF0D0A0000000010D0020432
:10C39000AAAA00006CEA0202CCCC0000BBBB0000E1
:10C3A0004F5441C9FDBCB6C6F4B6AF0D0A0000003B
:10C3B000CDF8C2E7C9FDBCB6C6F4B6AFC6F4B6AF99
:10C3C0000D0A000000A00004FFFF0000B4AEBFDAB9
:10C3D000C9FDBCB6C6F4B6AF0D0A0000014800683E
:10C3E0007047C0460C00004001218140044A1F28CC
:10C3F00002D01068884310601068084310607047CE
:10C400001C00004000480047C1A0020210B5401EB9
:10C4100007494860FF200006064A1368834303204B
:10C4200084071B19136000228A60086010BDC04693
:10C4300010E000E020ED00E080B50020FEF726FFD0
:10C44000404280BDB0B586B06C460F4918222046E8
:10C45000FDF756FE002528462146FEF71DFF0399ED
:10C460002846FEF77FFF0198012801D0082400E04C
:10C470000424002800D104460220FEF7D3FDE0404A
:10C480000249086006B0B0BD74CB020264F2020239
:10C49000F8B504460325002801D0284600E0042012
:10C4A0004D430C4E7719B978FEF7F8FD48206043EC
:10C4B000E8490958CA68802310461843C860705D6F
:10C4C0007C7824022018C8629A43CA60FEF73BFEBB
:10C4D000F8BDC0468CCB0202F8B50C460078DD4EA4
:10C4E000F168814209D0726D824206D0B168814202
:10C4F00012D0326D82420FD0F8BD0D1A681E8541F0
:10C500000095482068433018032C15D1876B102103
:10C51000284600F04FFA19E00D1A681E8541009573
:10C52000482068433018032C19D1C169002921D053
:10C530001C3000210160F8BD81691830302902D01B
:10C540000168102901D1802101600027482068433B
:10C5500030180021816301628162243017E0816913
:10C560001830302902D00168202901D180210160D2
:10C57000002704E0C76B2021284600F01BFA482062
:10C58000684330180021C163C1624163303000212B
:10C590000160002FB0D068462146B847F8BDC046BC
:10C5A000FEB50290482215464543AA494B59DE691B
:10C5B0000F2434404E19357C002D1FD04F214902E5
:10C5C0005A690A4249D0996904229143996102212A
:10C5D0001962012189076418F461F56B202100F0CC
:10C5E000E9F90020F063F0627063303600203060BB
:10C5F000002D36D002A82146A847FEBD0C2C30D80D
:10C600007C4424796400A744432C452C062C7F816C
:10C610002C2C2C2C0600B369202B03D01836336841
:10C62000302B1ED104461046134601946343CD18A7
:10C630002C6B2F4634376E6BA6420A4612D2D65860
:10C64000716909070ED5746839684B1C3B60EB6A49
:10C650005C54029C11460246E5E70C2CB3D0012C39
:10C66000B1D0FEBD3968A142FBD12E463036D1583B
:10C670008A6905239A438A61E86B0090202101981A
:10C6800000F098F90024EC63EC62009D3C60ADE79B
:10C6900001203CE008241C62B469102C04D034460C
:10C6A00018342468302CDCD1746AB56AA54213D1E1
:10C6B00035462435374628379969022291439961D6
:10C6C000B16B0091102100F075F90024B46334625D
:10C6D0003C602E46009D89E750430B189D6AA54299
:10C6E000BFD2064608584469A407BAD51C46283468
:10C6F00025686E1C26601B6A5B5D0360029813460A
:10C700004343CB185C6AE7E7022000E0042018628C
:10C71000FEBDC046FEB50E460546022803D3002ED8
:10C7200001D1012494E0002D03D0012D08D109246A
:10C7300000E008242046FEF757FC2046FFF754FE91
:10C74000482102956943BF4A505883691F240194C8
:10C75000A3438361062383600F230093036257186A
:10C760000024BC62BC63FC633C627C62FC623C6390
:10C77000317F3974727F7A74B27FBA747C63736864
:10C78000B268F56892002A435B1E032B0ED8C046A0
:10C790007B441B795B009F4401030507082304E0E9
:10C7A000182302E0282300E038231A433D461235BF
:10C7B000C260C907090F72699201D2B28918B269C1
:10C7C0009207920E8918491C8160796131690129AB
:10C7D00001D12221016131680298FFF759FE2878C2
:10C7E000002809D1384611300078002804D1384695
:10C7F00010300078002829D07868002816D403214A
:10C8000002468A43154953588507ED0EFF26AE4070
:10C81000B3438026AE401E4356500199014001208B
:10C820008840BF490860BF4908600FE08107C90E12
:10C83000FF228A40009D0540083D032085430648AD
:10C840002B58934380228A401A432A500120B86112
:10C850002046FEBD54E902021CED00E000E400E0C9
:10C86000F0B58DB005460C900120002900D19DE067
:10C870001646002A00D199E01C460F461021284692
:10C8800000F0B2F8002800D090E048231846684332
:10C890006C4922460C1800210291A162A263276212
:10C8A0006662217C0029039308D004A8142101901A
:10C8B000FDF73FFC012D1DD018201CE0A17C0029B4
:10C8C00036D0604F5D43785979198A6AB2422AD2CC
:10C8D0004269920727D50A46283213685C1C146007
:10C8E000096AC95C039B01600C9D184668433818AF
:10C8F000466AE7E71A200B90029D0A9502200990EC
:10C90000E0680199FEF72EFC0C98039941434D48CD
:10C9100042584018C0682649009139463346FEF710
:10C920008FFC284642E0816982220A4382613CE012
:10C930004449085881690A0602D5802291438161E1
:10C94000002702973F4A1946694350585418A16A74
:10C95000B1421DD247694F2149020F4212D14169AC
:10C96000890709D5214628310A68531C0B60039BAF
:10C97000216A895C01600C9D18466843314A101891
:10C98000466AE0E7022101620121029189070F4313
:10C99000416A0029FCD11021284600F00BF8A26B57
:10C9A000002A02D00CA83946904702980DB0F0BD7D
:10C9B000D9C4020210B50123EFF310821A4002D14C
:10C9C000EFF3108472B6482444431E48001984696A
:10C9D0008C4384618169002901D118300360002AE9
:10C9E00000D162B610BDC046B0B502460120EFF3DB
:10C9F0001083034002D1EFF3108472B648245443ED
:10CA0000104A12199569002D18D0802D16D01832B1
:10CA10000024102D09D0202D0BD0302D07D0402D13
:10CA20000CD0012D09D1116007E0202903D002208C
:10CA300004E01029FBD1302010602046002B00D1EB
:10CA400062B6B0BD54E90202B0B5002801D001249D
:10CA500018E0032081023D4802683D4B53500024FA
:10CA6000946001225303084D2B60BFF34F8FBFF337
:10CA70006F8F2B4D2B6003685A50847204811020F5
:10CA8000FEF7AAFA2046B0BD80E100E0F8B50C46FA
:10CA900001460120002902D0002C00D1F8BD6379A5
:10CAA000227915461D43F9D00F012848C619B372E3
:10CAB0007272A068F06010252846FEF795FA2846A5
:10CAC000FFF792FC2148C2590320810220485050B0
:10CAD000206810600020D06033460A33747A002C3E
:10CAE00003D094680225254395601B78002B0ED057
:10CAF000FF221202094B1C6894430122D5036419DA
:10CB00001C605203064B1A60064B1A603268936829
:10CB100001242343936054503472F8BD0CE400E0C8
:10CB200080E200E000E100E00146012000290CD194
:10CB300006490A7A002A08D00320820209680448BC
:10CB400088500020C86001238B507047E4E902023E
:10CB500051E5CC1A02E008C8121F08C1002AFAD118
:10CB600070477047002001E001C1121F002AFBD16D
:10CB700070470000000000000000000001000000FD
:10CB8000FFFFFFFF00000000000000005906201416
:10CB9000032145012882003241003219004113006F
:10CBA000390300B506002D03002D020022010022EA
:10CBB00001003E0100200000000000000000000015
:10CBC0000000000000000000000000000200000063
:10CBD0000000000014000000020000000700000038
:10CBE000020000000200000000000000020000003F
:10CBF000000000001400000002000000010000001E
:10CC0000020000000200000002000000000000001E
:10CC100014000000000000000700000000000000F9
:10CC20000000000003000000000000000000000001
:10CC300000000000010000000000000000000000F3
:10CC40000200000004000000001003EB00000000E0
:10CC5000010000000100000004000000000100329B
:10CC600000000000000000000000000001000000C3
:10CC700001000005000000000000000000000000AE
:10CC8000010000000100003500000000010000006C
:10CC90000000000004000000000000200000000070
:10CCA000010000000000000004000000000000D8A7
:10CCB0000000000001000000000000000100000072
:10CCC000000000060000000001000000000000005D
:10CCD0000100000002000001000000000000000050
:10CCE00000000000010000000300009F00000000A1
:10CCF000010000000000000001000000000000B979
:10CD00000000000001000000000000000100000021
:10CD1000000000AB210504198912130018DECA01B6
:10CD2000305201231305331993070800205BA34AEF
:10CD300021BAF9FC0A0A0D2050726F6772616D6D9D
:10CD4000696E6720436F6D706C6574656420537500
:10CD5000636365737366756C6C79210A0D2D2D2DD7
:10CD60002D2D2D2D2D2D2D2D2D2D2D2D2D2D2D2DF3
:10CD70002D2D2D2D2D2D2D2D2D2D2D2D2D0D0A2033
:10CD80004E616D653A200000A8CD020200E8020263
:10CD9000F40100006CA1020208CE0202F4E90202D2
:10CDA000780D000064CB0202520332805201342617
:10CDB000B803350F0001014521AD020203455006BD
:10CDC000C570014013D6207001401445B000500BCF
:10CDD0004202820345FFFF0F203204420832010461
:10CDE000561000010551200050074590014018429F
:10CDF00004023D0545A00140194206023D07454099
:08CE000001400D820100000059
:020000040202F6
:10CFA000A5A54B4D0000001000000002AAAA5A7F60
:10CFB000A0CF0202000000000200000000000000FC
:10CFC0000000000000000000000000000000000061
:10CFD0000000000000000000000000000000000051
:10CFE00038D00202000000000A56656E646F7209B4
:10CFF0003A204D4B53454D490A43686970093A2020
:10D000004D4B383030300A44617465093A204D6127
:10D010007220203520323032350A56657273696FBE
:10D020006E093A2056302E362E32000000000000E5
:08D030000000000000000000F8
:040000050202A0C192
:00000001FF
